:0200000480007A
:100000006F008004732F2034930F80006308FF0378
:10001000930F90006304FF03930FB0006300FF038E
:10002000130F000063040F0067000F00732F2034CC
:1000300063540F006F00400093E19153171F0000BD
:1000400023223FFC6FF09FFF93000000130100008C
:10005000930100001302000093020000130300004C
:100060009303000013040000930400001305000034
:10007000930500001306000093060000130700001C
:100080009307000013080000930800001309000004
:1000900093090000130A0000930A0000130B0000EC
:1000A000930B0000130C0000930C0000130D0000D4
:1000B000930D0000130E0000930E0000130F0000BC
:1000C000930F0000732540F16310050097020000B4
:1000D000938202017390523073500018970200000F
:1000E0009382020273905230B70200809382F2FF33
:1000F0007390023B9302F0017390023A73504030C8
:100100009702000093824201739052307350203066
:100110007350303093010000970200009382C2EECA
:1001200073905230130510001315F501634C050050
:100130000F00F00F930110009308D0051305000085
:100140007300000093020000638A02007390521053
:10015000B7B2000093829210739022307350003037
:10016000970200009382420173901234732540F18C
:1001700073002030B70001FF938000F037110F0F9C
:100180001301F1F033E72000B70310FF9383F3F07E
:10019000930120006312774AB710F00F938000FF9D
:1001A00037F1F0F01301010F33E72000B703F1FF3F
:1001B000938303FF9301300063107748B700FF007B
:1001C0009380F00F37110F0F1301F1F033E7200088
:1001D000B713FF0F9383F3FF93014000631E77442F
:1001E000B7F00FF09380F00037F1F0F01301010F3A
:1001F00033E72000B7F3FFF09383F30F9301500030
:10020000631C7742B70001FF938000F037110F0F96
:100210001301F1F0B3E02000B70310FF9383F3F074
:1002200093016000639A7040B70001FF938000F073
:1002300037110F0F1301F1F033E12000B70310FF66
:100240009383F3F0930170006318713EB70001FFD0
:10025000938000F0B3E01000B70301FF938303F035
:1002600093018000639A703C13020000B70001FF05
:10027000938000F037110F0F1301F1F033E72000E6
:10028000130307001302120093022000E31052FE32
:10029000B70310FF9383F3F093019000631E73384C
:1002A00013020000B710F00F938000FF37F1F0F059
:1002B0001301010F33E720001300000013030700B0
:1002C0001302120093022000E31E52FCB703F1FF59
:1002D000938303FF9301A0006310733613020000A1
:1002E000B700FF009380F00F37110F0F1301F1F0EB
:1002F00033E7200013000000130000001303070081
:100300001302120093022000E31C52FCB713FF0FEC
:100310009383F3FF9301B000631073321302000064
:10032000B70001FF938000F037110F0F1301F1F0B8
:1003300033E720001302120093022000E31252FE62
:10034000B70310FF9383F3F09301C0006316772E79
:1003500013020000B710F00F938000FF37F1F0F0A8
:100360001301010F1300000033E7200013021200F5
:1003700093022000E31052FEB703F1FF938303FFC3
:100380009301D000631A772A13020000B700FF0020
:100390009380F00F37110F0F1301F1F013000000DD
:1003A0001300000033E72000130212009302200024
:1003B000E31E52FCB713FF0F9383F3FF9301E0009A
:1003C000631C772613020000B70001FF938000F042
:1003D0001300000037110F0F1301F1F033E7200075
:1003E0001302120093022000E31052FEB70310FF25
:1003F0009383F3F09301F00063107724130200005D
:10040000B710F00F938000FF1300000037F1F0F0F9
:100410001301010F1300000033E720001302120044
:1004200093022000E31E52FCB703F1FF938303FF06
:10043000930100016312772013020000B700FF0050
:100440009380F00F130000001300000037110F0F0E
:100450001301F1F033E72000130212009302200091
:10046000E31E52FCB713FF0F9383F3FF93011001B8
:100470006314771C1302000037110F0F1301F1F002
:10048000B70001FF938000F033E720001302120051
:1004900093022000E31252FEB70310FF9383F3F0A0
:1004A00093012001631A77181302000037F1F0F06E
:1004B0001301010FB710F00F938000FF130000002D
:1004C00033E720001302120093022000E31052FED3
:1004D000B703F1FF938303FF93013001631E771489
:1004E0001302000037110F0F1301F1F0B700FF00E6
:1004F0009380F00F130000001300000033E720008A
:100500001302120093022000E31E52FCB713FF0FE8
:100510009383F3FF930140016310771213020000ED
:1005200037110F0F1301F1F013000000B70001FFA6
:10053000938000F033E720001302120093022000A2
:10054000E31052FEB70310FF9383F3F093015001C1
:100550006314770E1302000037F1F0F01301010F5E
:1005600013000000B710F00F938000FF130000008D
:1005700033E720001302120093022000E31E52FC16
:10058000B703F1FF938303FF930160016316770ABA
:100590001302000037110F0F1301F1F013000000D8
:1005A00013000000B700FF009380F00F33E7200036
:1005B0001302120093022000E31E52FCB713FF0F38
:1005C0009383F3FF9301700163187706B70001FF6F
:1005D000938000F033611000B70301FF938303F0B1
:1005E00093018001631A7104B700FF009380F00F3C
:1005F00033E10000B703FF009383F30F93019001F1
:10060000631C7102B3600000930300009301A0011A
:1006100063947002B71011119380101137212222B8
:100620001301212233E02000930300009301B00165
:1006300063147000631030020F00F00F638001003C
:100640009391110093E111009308D00513850100E7
:10065000730000000F00F00F930110009308D00505
:100660001305000073000000731000C000000000BC
:0C0670000000000000000000000000007E
:1010000000000000000000000000000000000000E0
:1010100000000000000000000000000000000000D0
:1010200000000000000000000000000000000000C0
:1010300000000000000000000000000000000000B0
:081040000000000000000000A8
:040000058000000077
:00000001FF
